:020000040000FA
:02000000CB280B
:08000800F100030EF000831665
:1000100003138C1E0F28831203138C1A28288316AF
:1000200003130C1E1728831203130C1AAE28831611
:1000300003130C1F1F28831203130C1B8A2883161B
:1000400003130C1C2728831203130C187928C628C5
:10005000831203131A08F20000307202031D3428C1
:100060009F121F129F11652801307202031D3C2848
:100070009F121F129F15652802307202031D44282B
:100080009F121F169F11652803307202031D4C2812
:100090009F121F169F15652804307202031D5428F5
:1000A0009F161F129F11652805307202031D5C28E0
:1000B0009F161F129F15652806307202031D6428C3
:1000C0009F161F169F11652872280C10F701F30167
:1000D000F401F5018F01831603130C14831203132B
:1000E0000C14722883120313981CC62818121816B1
:1000F000C628F70A101066308E0703188F0AF830EA
:100100008F0710149E3081000B110B1D85281F15C1
:100110000C10C628F03081000B110B1D8D281E0815
:10012000F800831603131E08F900831203137908DD
:10013000F50703189C289F28F40A0319F30A780886
:10014000F4070318F30A0C13F708031DC6288316D7
:1001500003130C160C1083120313C628F60A013081
:100160007602031DB628730899000F280230760224
:10017000031DBD28740899000F287508990083167F
:1001800003130C1283120313F601C628700E8300AA
:10019000F10E710E09008312031385018601831687
:1001A0000313D8308100FF308500FF3086007F3098
:1001B0009B001F129F129F171F13831203139F1779
:1001C0001F13831603138130990024309800831283
:1001D00003139030980085018601F601F7010C1396
:1001E000831603138C160C120C170B178B17831224
:1001F00003131F149012101290101014FF28FF28E0
:02400E00623F0F
:02401000FC3F73
:00000001FF
